:107C0000112404B714BE01FD07C003FD27D18CB5B4
:107C10008F7A8CBD802FEAD185E08093810082E04D
:107C20008093C00088E18093C10086E08093C20009
:107C300080E18093C4008EE0FBD0219A84E028E1AB
:107C40003EEF91E0309385002093840096BBB09B7B
:107C5000FECF199AA8958150A9F7EE24FF24AA24F3
:107C6000A394B5E0CB2EA1E1BA2EF3E0DF2ED2D063
:107C7000813461F4CFD0082FE1D0023829F10138E6
:107C800011F485E001C083E0BDD07FC0823411F4DF
:107C900084E103C0853419F485E0D8D076C08535F9
:107CA00079F4B8D0E82EFF24B5D0082F10E0102FBB
:107CB00000270E291F29000F111FC0D0780165C0B1
:107CC000863521F484E0C2D080E0DECF843609F02E
:107CD00040C0A0D09FD0082F9DD080E0E81680E75C
:107CE000F80618F4F701D7BEE895C0E0D1E092D0CD
:107CF00089930C17E1F7F0E0EF16F0E7FF0618F0B4
:107D0000F701D7BEE8959AD007B600FCFDCFA701D2
:107D1000A0E0B1E02C9130E011968C91119790E0A9
:107D2000982F8827822B932B1296FA010C01A7BE5D
:107D3000E89511244E5F5F4FF1E0A038BF0751F77F
:107D4000F701C7BEE89507B600FCFDCFB7BEE895C2
:107D50001CC0843761F45ED05DD0082F5BD06ED03C
:107D6000F70185917F014ED00150D1F70EC08537C4
:107D700039F464D08EE146D085E944D08FE084CFD9
:107D8000813511F488E054D059D080E13BD06FCFD9
:107D90008EBD0DB407FEFDCF8EB50895289885E001
:107DA000F7DF80E0F5DF289A817008951F93182F80
:107DB000662321F086E060E0F9DF289AEFDF882370
:107DC000E9F72898812FE4DF1F910895EF92FF9241
:107DD0000F931F937B018C0183E060E0E7DFC80114
:107DE000AA27BB27D5DFBB27A12F902F8F2DD0DF50
:107DF0008E2DCEDF80E0CCDF289A1F910F91FF906F
:107E0000EF900895982F8091C00085FFFCCF90934C
:107E1000C6000895199A8091C00087FFFCCF809119
:107E2000C00084FD01C0A8958091C600199A0895EC
:107E3000E0E6F0E098E1908380830895EBDF803204
:107E400019F088E0F5DFFFCF84E1DCCF1F93182F16
:107E5000E1DF1150E9F7F2DF1F9108959F92AF9291
:107E6000BF92CF92DF92EF92FF920F931F93CF9327
:107E7000DF9380E0DDDF84B18D6284B9289A2A9A8D
:107E80008CB580658CBD28988FE982DF80E080DF2B
:107E9000289A81508E3F08F09DC081E061E086DF26
:107EA00080E076DF289A60E070E080E090E08EDF8E
:107EB000863409F08FC061E070E080E090E086DFFA
:107EC0008C3409F087C062E070E080E090E07EDFF3
:107ED000883509F07FC066E070E080E090E076DFF2
:107EE0008A3309F077C069E070E080E090E06EDFEF
:107EF0008A3309F06FC067E070E080E090E066DFF1
:107F0000082F68E070E080E090E060DF10E0F02E85
:107F1000EE2490E0E82AF92AE0FC5CC0199AC0E05F
:107F2000D0E0CC24DD249924939443E0A42E35E0C2
:107F3000B32E30C02A96BE0180E090E047DF082FC4
:107F400010E02196BE0180E090E02B973FDF90E0AB
:107F5000982F8827802B912BFE010C0197BEE89566
:107F600011242296CE018F779070892B19F0CE15AF
:107F7000DF0581F4F601A7BEE89507B600FCFDCF4A
:107F8000F601B7BEE89507B600FCFDCF80E890E0AB
:107F9000C80ED91ECE15DF0508F4CCCF199881E1A3
:107FA00087BFE895EAE0F0E0EE0EFF1EF1E0EF1685
:107FB000F0E8FF0610F482E501C088ED61E0F6DE2E
:107FC00080E0E6DE80E0E4DE80E0E2DE289A88E021
:107FD0002FDFFFCFDF91CF911F910F91FF90EF9097
:107FE000DF90CF90BF90AF909F900895282E80E0B3
:087FF0001FDFEE27FF270994B3
:027FFE0000057C
:0400000300007C007D
:00000001FF
